:100000000C9462000C948A000C948A000C948A0070
:100010000C948A000C948A000C948A000C948A0038
:100020000C948A000C948A000C948A000C948A0028
:100030000C948A000C948A000C948A000C948A0018
:100040000C948F030C948A000C9405050C948A0080
:100050000C948A000C948A000C948A000C948A00F8
:100060000C948A000C948A000000000024002700F1
:100070002A0000000000250028002B0000000000DE
:1000800023002600290004040404040404040202DA
:100090000202020203030303030301020408102007
:1000A0004080010204081020010204081020000012
:1000B0000007000201000003040600000000000029
:1000C00000004E0611241FBECFEFD8E0DEBFCDBF2B
:1000D00011E0A0E0B1E0E4E9FEE002C005900D927D
:1000E000A831B107D9F711E0A8E1B1E001C01D9234
:1000F000A13FB107E1F710E0C4ECD0E004C02297C3
:10010000FE010E944407C23CD107C9F70E94880340
:100110000C9448070C940000CF92DF92FF920F934B
:100120001F93CF93DF93F82E062F142F862F61E0B5
:100130000E9449048F2D61E00E9449048F2D60E0E8
:100140000E946904802F60E00E946904C7E0D0E04B
:10015000C12EDD24802F60E00E946904B6010C2EC0
:1001600002C0759567950A94E2F761708F2D0E9421
:100170006904802F61E00E9469048F2D60E00E9475
:10018000690421978FEFCF3FD80721F7802F60E0D8
:100190000E946904DF91CF911F910F91FF90DF9032
:1001A000CF900895CF92DF92EF92FF920F931F931B
:1001B000CF93DF936C01C0E0D0E07B010027F7FC18
:1001C0000095102F79C08091000160E00E946904C1
:1001D00060910201709103018091040190910501E9
:1001E00040911B010E948C006091020170910301FB
:1001F0008091040190910501409125010E948C009D
:1002000060910201709103018091040190910501B8
:1002100040912F010E948C006091020170910301B6
:100220008091040190910501409139010E948C0058
:100230008091000161E00E946904C801B7010E9439
:10024000E5038091000160E00E9469046091020171
:1002500070910301809104019091050140E00E949A
:100260008C006091020170910301809104019091D2
:10027000050140E00E948C00609102017091030131
:10028000809104019091050140E00E948C006091F2
:10029000020170910301809104019091050140E0F9
:1002A0000E948C008091000161E00E946904C801F5
:1002B000B7010E94E5032196CC15DD050CF483CF30
:1002C000DF91CF911F910F91FF90EF90DF90CF9032
:1002D0000895CF92DF92EF92FF920F931F93CF93E7
:1002E000DF936C01C0E0D0E07B010027F7FC0095B4
:1002F000102F75C08091000160E00E946904609138
:1003000002017091030180910401909105014FEF6A
:100310000E948C00609102017091030180910401A0
:10032000909105014FEF0E948C0060910201709145
:10033000030180910401909105014FEF0E948C0010
:100340006091020170910301809104019091050177
:100350004FEF0E948C008091000161E00E946904CF
:10036000C801B7010E94E5038091000160E00E948E
:1003700069046091020170910301809104019091E0
:10038000050140E00E948C00609102017091030120
:10039000809104019091050140E00E948C006091E1
:1003A000020170910301809104019091050140E0E8
:1003B0000E948C0060910201709103018091040100
:1003C0009091050140E00E948C008091000161E065
:1003D0000E946904C801B7010E94E5032196CC156B
:1003E000DD050CF487CFDF91CF911F910F91FF9026
:1003F000EF90DF90CF900895EF92FF920F931F93AD
:10040000E0900601F09007010091080110910901A8
:100410008091000160E00E94690420910201309106
:100420000301C8016AE070E00E94DE06FB01E55EA0
:10043000FE4F8091040190910501B90140810E9415
:100440008C00809106019091070162E070E00E94AB
:10045000DE069C012D5B3E4FC8016AE070E00E9401
:10046000DE06FC01EB5DFE4FD9014C918081482BEB
:1004700040931A016091020170910301809104017F
:10048000909105010E948C0020910201309103019E
:10049000C7016AE070E00E94DE06FB01E15DFE4FED
:1004A0008091040190910501B90140810E948C0066
:1004B0002091020130910301C7016AE070E00E94BF
:1004C000DE06FC01E75CFE4F80910401909105017E
:1004D000B90140810E948C008091000161E00E947E
:1004E00069041F910F91FF90EF90089580910A0188
:1004F0000E94B604892B81F0109219011092180104
:100500008CE290E0909307018093060187E090E0F1
:1005100090930901809308010E94D70320914D0117
:1005200030914E0140914F0150915001621B730B6D
:10053000840B950B685E734080409040D8F08091AA
:10054000180190911901892BA9F40E94D703609397
:100550004D0170934E0180934F01909350010E9482
:10056000FC0180910601909107010197909307018A
:1005700080930601809106019091070197FF0FC0BB
:10058000809108019091090101979093090180934E
:1005900008018BE390E0909307018093060180911E
:1005A00008019091090197FF10C081E090E09093BD
:1005B000190180931801109209011092080185E039
:1005C00090E068EE73E00E94D200089580910001EF
:1005D00061E00E94490480910A0160E00E944904A0
:1005E00080910C0161E00E9449048EED91E040E0B1
:1005F00051EE60E070E00E94420580910C0160E0E5
:100600000E9469048FE680931B0183E080931C01A4
:10061000FDE5F0931D0187E580931E0183E3809340
:100620001F0186E7809320018EE78093210183E4F8
:1006300080932201EFE7E093230177E77093240191
:100640001092430181E08093440110924501809310
:10065000460110924701809348011092490180930E
:100660004A0110924B0180934C018EED809325013D
:1006700086E0809326018AEB809327018EEA80939F
:10068000280196E6909329018CEE80932A018CEF45
:1006900080932B0186E880932C018EEF80932D01AF
:1006A0008EEE80932E016BE760932F0150E65093FE
:1006B0003001F093310145E74093320190933301CB
:1006C00037E3309334012FE32093350181E68093A3
:1006D0003601E093370170933801609339015093EC
:1006E0003A01F0933B0140933C0190933D013093DC
:1006F0003E0120933F0180934001E09341017093BC
:10070000420182E090E064EF71E00E946901089587
:100710000E940F040E94E6020E947602FDCF1F9203
:100720000F920FB60F9211242F933F938F939F93A5
:10073000AF93BF938091550190915601A0915701BD
:10074000B0915801309159010196A11DB11D232F7F
:100750002D5F2D3720F02D570196A11DB11D20933F
:1007600059018093550190935601A0935701B0937E
:1007700058018091510190915201A0915301B09183
:1007800054010196A11DB11D809351019093520116
:10079000A0935301B0935401BF91AF919F918F915A
:1007A0003F912F910F900FBE0F901F9018958FB70C
:1007B000F894209155013091560140915701509184
:1007C00058018FBFB901CA010895EF92FF920F93AC
:1007D0001F937B018C018FB7F89440915501509184
:1007E000560160915701709158018FBF2FB7F8944F
:1007F0008091550190915601A0915701B0915801F7
:100800002FBF841B950BA60BB70BE816F9060A073A
:100810001B0760F71F910F91FF90EF900895789458
:1008200084B5826084BD84B5816084BD85B58260F5
:1008300085BD85B5816085BDEEE6F0E08081816093
:100840008083E1E8F0E08081826080838081816044
:100850008083E0E8F0E0808181608083E1EBF0E07C
:10086000808184608083E0EBF0E080818160808320
:10087000EAE7F0E080818460808380818260808309
:100880008081816080838081806880831092C10034
:100890000895282F30E0C90186569F4FFC0194919E
:1008A0002A573F4FF9018491882391F0E82FF0E017
:1008B000EE0FFF1FE859FF4FA591B491662329F46D
:1008C0008C91909589238C9308958C91892B8C938E
:1008D0000895482F50E0CA0182559F4FFC01249192
:1008E000CA0186569F4FFC0194914A575F4FFA0107
:1008F00034913323D1F1222331F1233021F480913B
:1009000080008F7705C0243031F4809180008F7D86
:100910008093800018C0213019F484B58F7704C00B
:10092000223021F484B58F7D84BD0DC0263021F4A2
:100930008091B0008F7705C0273029F48091B000F6
:100940008F7D8093B000E32FF0E0EE0FFF1FEE5895
:10095000FF4FA591B491662329F48C91909589233A
:100960008C9308958C91892B8C930895682F70E057
:10097000CB0182559F4FFC012491CB0186569F4F9E
:10098000FC0144916A577F4FFB019491992319F41C
:1009900020E030E038C0222331F1233021F480916F
:1009A00080008F7705C0243031F4809180008F7DE6
:1009B0008093800018C0213019F484B58F7704C06B
:1009C000223021F484B58F7D84BD0DC0263021F402
:1009D0008091B0008F7705C0273029F48091B00056
:1009E0008F7D8093B000892F90E0880F991F8458E5
:1009F0009F4FFC01A591B4918C9120E030E08423BD
:100A000011F021E030E0C90108951F920F920FB656
:100A10000F9211242F933F934F935F936F937F9384
:100A20008F939F93AF93BF93EF93FF934091C60033
:100A3000E091DA01F091DB01CF01019660E870E00E
:100A40000E94DE069C018091DC019091DD01281757
:100A5000390739F0E65AFE4F40833093DB0120938B
:100A6000DA01FF91EF91BF91AF919F918F917F91AB
:100A70006F915F914F913F912F910F900FBE0F900B
:100A80001F9018955F926F927F928F929F92AF9274
:100A9000BF92CF92DF92EF92FF920F931F93CF936B
:100AA000DF93EC013A014B01413482E458078FE0B7
:100AB000680780E078070CF07FC060E874E88EE19A
:100AC00090E0A40193010E94130721503040404060
:100AD0005040CA01B90122E030E040E050E00E94FD
:100AE000130759016A01A60195012095309540959B
:100AF000509594E0220F331F441F551F9A95D1F74C
:100B000060E074E284EF90E00E941307CA01B9012B
:100B10002FEF30E040E050E00E94BF06A4019301B7
:100B20000E941307C90181509F4F181619061CF423
:100B3000522E5A9403C055245394521A60E079E01F
:100B40008DE390E0A40193010E94130721503040EF
:100B500040405040CA01B90122E030E040E050E09E
:100B60000E941307209530954095509583E0220F01
:100B7000331F441F551F8A95D1F760E074E284EF5C
:100B800090E00E941307CA01B9012FEF30E040E066
:100B900050E00E94BF06A40193010E941307C901FF
:100BA00081509F4F181619061CF4822F815002C0E5
:100BB00081E0821B851500F5E885F98581E090E0EC
:100BC0000A8802C0880F991F0A94E2F7808360E0C8
:100BD00079E08DE390E0A40193010E941307215076
:100BE000304040405040CA01B90122E030E040E0CE
:100BF00050E00E94130704C0E885F9851082950132
:100C0000EC81FD813083EE81FF812083EA85FB85C5
:100C1000208141E050E0CA010E8402C0880F991F74
:100C20000A94E2F7282B2083EA85FB852081CA01FC
:100C30000F8402C0880F991F0A94E2F7282B2083A3
:100C4000EA85FB858081088802C0440F551F0A94FD
:100C5000E2F7842B8083DF91CF911F910F91FF905A
:100C6000EF90DF90CF90BF90AF909F908F907F904C
:100C70006F905F900895FC01A085B18521898C91CA
:100C800090E0022E02C0959587950A94E2F780FFC6
:100C9000F6CF0484F585E02D6083089582E191E02C
:100CA0009093DF018093DE018AE591E09093E1016A
:100CB0008093E00185EC90E09093E3018093E20162
:100CC00084EC90E09093E5018093E40180EC90E067
:100CD0009093E7018093E60181EC90E09093E90125
:100CE0008093E80186EC90E09093EB018093EA0119
:100CF00084E08093EC0183E08093ED0187E08093B2
:100D0000EE0185E08093EF0181E08093F00108958A
:100D10000F931F93CF93DF938C01EB0109C02196B2
:100D2000D801ED91FC910190F081E02DC801099569
:100D300068816623A1F7DF91CF911F910F910895EC
:100D4000EF92FF920F931F93CF93DF938C017B0160
:100D5000EA010CC0D7016D917D01D801ED91FC91A4
:100D60000190F081E02DC80109952197209791F716
:100D7000DF91CF911F910F91FF90EF900895629FA7
:100D8000D001739FF001829FE00DF11D649FE00D83
:100D9000F11D929FF00D839FF00D749FF00D659FE4
:100DA000F00D9927729FB00DE11DF91F639FB00DE3
:100DB000E11DF91FBD01CF011124089597FB092EF4
:100DC00007260AD077FD04D049D006D000201AF4B7
:100DD000709561957F4F0895F6F7909581959F4F97
:100DE0000895A1E21A2EAA1BBB1BFD010DC0AA1F6C
:100DF000BB1FEE1FFF1FA217B307E407F50720F084
:100E0000A21BB30BE40BF50B661F771F881F991FFE
:100E10001A9469F760957095809590959B01AC0147
:100E2000BD01CF01089597FB092E05260ED057FD71
:100E300004D0D7DF0AD0001C38F450954095309587
:100E400021953F4F4F4F5F4F0895F6F7909580954E
:100E5000709561957F4F8F4F9F4F0895AA1BBB1BC5
:100E600051E107C0AA1FBB1FA617B70710F0A61BAA
:100E7000B70B881F991F5A95A9F780959095BC01CB
:100E8000CD010895EE0FFF1F0590F491E02D099418
:040E9000F894FFCF04
:100E940008000C000B003B000E00060007000000D9
:080EA40000003B068806A006D1
:00000001FF
